:100000000C94AA020C9441240C94C7020C94C702CD
:100010000C94C7020C94C7020C94C7020C94C7023C
:100020000C94C7020C94C7020C94602B0C94322CD5
:100030000C944B260C94C7020C94C7020C94C70274
:100040000C94C7020C94C7020C94C7020C94C7020C
:100050000C94C7020C94EF260C94C7020C94C702B0
:100060000C94C7020C94C7020C94C7020C94C702EC
:100070000C94C7020C94C7020C94C7020C94C702DC
:100080000C94C7020C94C7020C94C7020C94C702CC
:100090000C94C7020C94C7020C94C7020C94C702BC
:1000A0000C94C7020C94C7020C94C7028305830505
:1000B000AF05AF05170635064D074D074006D906B3
:1000C000EA06EA069F2CC62CBE2DC62CBE2D122D8C
:1000D000352DBE2D8C2D9B2D29001E001F002000CC
:1000E0002100220000002B0014001A000800150057
:1000F00017009141E00004001600070009000A0003
:100100000000E1001D001B000600190005000000B2
:10011000296434002D002E002800E3002C002A0062
:1001200027002600250024002300000031003800AD
:10013000130012000C0018001C00280033000F00F0
:100140000E000D000B000000E50037003600100027
:100150001100904100004F00520051005000015129
:100160004C00286735003A003B003C003D003E0053
:100170000000010034023400350025022E022E005A
:1001800001001F023302350001002D0000000100B4
:1001900000000000000037003800000001000100EE
:1001A00001000100010001000100010043004200C4
:1001B000410040003F000000890023023502250273
:1001C00031022702260201002D00380037003000DE
:1001D0002F00000001003800370030022F0201001C
:1001E0000000370223022D02360201000100010047
:1001F00000047F3F1F643214643214783C1E1E14C6
:100200000A052223252628292A2C2D2F3032333582
:1002100036383A3B3D3E4042434547494A4C4E50B2
:1002200051535557595A5C5E6062646668696B6DDC
:100230006F71737577797B7D7F81838587898A8CE0
:100240008E90929496989A9C9E9FA1A3A5A7A8AAE7
:10025000ACAEAFB1B3B4B6B8B9BBBCBEBFC1C2C31C
:10026000C5C6C7C9CACBCCCDCED0D1D2D2D3D4D5B6
:10027000D6D7D7D8D9D9DADADBDBDBDCDCDCDCDCDF
:10028000DDDDDDDDDCDCDCDCDCDBDBDBDADAD9D9B7
:10029000D8D7D7D6D5D4D3D2D2D1D0CECDCCCBCA45
:1002A000C9C7C6C5C3C2C1BFBEBCBBB9B8B6B4B36B
:1002B000B1AFAEACAAA8A7A5A3A19F9E9C9A989601
:1002C0009492908E8C8A89878583817F7D7B7977D4
:1002D0007573716F6D6B6968666462605E5C5A59B4
:1002E00057555351504E4C4A4947454342403E3D75
:1002F0003B3A3836353332302F2D2C2A2928262503
:100300002322FFAA7F5540000101010101010101E3
:1003100001020202020202020202030303030303B8
:100320000303040404040404040505050505060686
:100330000606060707070707080808080909090944
:100340000A0A0A0B0B0B0C0C0C0D0D0D0E0E0E0FEA
:100350000F0F10101111111212131314141515167A
:10036000161717181819191A1A1B1B1C1D1D1E1EEB
:100370001F2020212222232424252626272829293C
:100380002A2B2C2D2D2E2F30313232333435363767
:1003900038393A3B3C3D3E3F404142434445464765
:1003A00048494A4C4D4E4F50515354555658595A3E
:1003B0005B5D5E5F616264656668696B6C6D6F70E2
:1003C00072737577787A7B7D7E8082838587888A51
:1003D0008C8E8F91939596989A9C9EA0A2A3A5A788
:1003E000A9ABADAFB1B3B5B7BABCBEC0C2C4C6C984
:1003F000CBCDCFD1D4D6D8DBDDDFE2E4E7E9EBEE3D
:10040000F0F3F5F8FAFDFF260354006800650020BC
:10041000004B00750064006F00780020004B006501
:1004200000790062006F0061007200640000001635
:10043000034B0075006D0061006F0020004B006FE2
:100440000062006F0000000403090409023B00027F
:100450000100A0FA090400000103010100092111B3
:100460000100012240000705810308000109040181
:10047000000103000000092111010001227B000797
:100480000582032000011201000200000008BAAB3F
:10049000909600010102000105010902A1018502F7
:1004A0000901A10005091901290815002501950870
:1004B000750181020501093009311581257F9502F9
:1004C0007508810609381581257F95017508810613
:1004D000050C0A38021581257F950175088106C033
:1004E000C005010980A101850319012AB700150182
:1004F00026B700950175108100C0050C0901A10106
:10050000850419012AA002150126A0029501751083
:100510008100C005010906A101050719E029E715B9
:100520000025019508750181029501750881010575
:1005300007190029FF150026FF00950675088100A0
:1005400005081901290595057501910295017503A5
:100550009101C00011241FBECFEFDAE0DEBFCDBF96
:1005600011E0A0E0B1E0E8E1FEE502C005900D92E7
:10057000A83DB107D9F723E0A8EDB1E001C01D9275
:10058000A832B207E1F70E9413160C940A2F0C94BC
:10059000000081E0089581E008950C94CB02089555
:1005A0000C94CF021F93CF93DF9300D000D01F9203
:1005B000CDB7DEB749835A836B833091DB018981E4
:1005C0009A81311114C0662359F0222349F00E9408
:1005D0008A09182F682F89819A810E94330903C0E4
:1005E0000E945E09182F69817A81812F04C00E94C0
:1005F0008A0969817A810F900F900F900F900F9068
:10060000DF91CF911F910C94B110FC01262F4081F6
:1006100051816281738184810C94D20281E00895BA
:10062000CF93DF93EC0160E00E940503BE01DF91F0
:10063000CF910C94D0020C9427120C94231208959D
:100640000E94DD070E941F032FEF84E39CE02150EE
:1006500080409040E1F700C000000C9415270F93F4
:100660001F93CF93DF938C0161E00E940503EC019F
:10067000B8010E94CD02882309F444C0B801CE011C
:100680000E944E238823F1F1B801CE010E94ED1F94
:100690008823C1F1B801CE010E94AA22882391F1DA
:1006A000B801CE010E94DB1E882361F1F80182812E
:1006B000882309F1CB358DE5D807C1F050F4C11579
:1006C000FCE5DF0781F0CF3DDC45A9F40E94BB0EBD
:1006D00019C0CC35EDE5DE0761F0CD35DD4559F4C7
:1006E0000E94040E08C00E9420030CC00E940D0E40
:1006F00002C00E94100EC801DF91CF911F910F918F
:100700000C94C90280E0DF91CF911F910F91089561
:100710000E942E260C94A1030E94A4030C9434265C
:1007200008950C94900381E008950C949303089528
:10073000CF93C82F0E9491038C2F0E949503CF91D5
:10074000089580E00C9498030E946C250C94980303
:100750000E946C259091DA01891721F08093DA01CB
:100760000C9498030895CF93DF93CDB7DEB72B9702
:100770000FB6F894DEBF0FBECDBF4F835887698791
:100780007A878B8761110E94500D9E012F5F3F4F2A
:1007900086E0F90111928A95E9F785E0FE01379626
:1007A000D90101900D928A95E1F789819A814C8156
:1007B0005D81452B31F09F3F31F491E08F3F19F47B
:1007C00003C091E001C090E090FF09C049815A81C7
:1007D0006B817C818D819E810E94710C05C0C90155
:1007E0000E940E038111F2CF2B960FB6F894DEBF54
:1007F0000FBECDBFDF91CF910895FC018081918123
:100800000E94CC090895CF93882309F4A9C0C82F6A
:100810008238C1F40E946C2581FDA2C069E38091F9
:100820000201909103010E9406260E94720D2FEF93
:1008300081EE94E0215080409040E1F700C000003C
:1008400069E319C0833801F50E946C2580FD88C0DA
:1008500063E580910201909103010E9406260E94A7
:10086000720D2FEF81EE94E0215080409040E1F72F
:1008700000C0000063E580910201909103010E9495
:100880000826CF910C94720D8438C1F40E946C2517
:1008900082FD66C067E480910201909103010E948D
:1008A00006260E94720D2FEF81EE94E021508040C9
:1008B0009040E1F700C0000067E4DDCF8CEF8C0FC3
:1008C000813AF8F48C2F0E946122811149C06C2F6B
:1008D00080910201909103010E94D025882349F064
:1008E0006C2F80910201909103010E9408260E94C2
:1008F000720D6C2F80910201909103010E940626D7
:10090000C0CF80E28C0F883048F4C77081E001C00E
:10091000880FCA95EAF70E94330DB3CFEBE5EC0FD1
:10092000E33040F4F0E0EF58FE4F808190E0CF914B
:100930000C949825E8E5EC0FE73150F4F0E0EE0F69
:10094000FF1FED5BFE4F80819181CF910C94AE250E
:10095000CD3E30F08C2F0E949816CF910C946A17E0
:10096000CF910895882309F464C0823879F40E94F5
:100970006C2581FF5EC069E38091020190910301C3
:100980000E9406260E94720D69E310C08338B1F4FC
:100990000E946C2580FF4DC063E58091020190911B
:1009A00003010E9406260E94720D63E580910201F8
:1009B000909103010E9408260C94720D843879F4FA
:1009C0000E946C2582FF35C067E4809102019091FE
:1009D00003010E9406260E94720D67E4E7CF9CEF98
:1009E000980F913A10F4682FE1CF90E2980F983069
:1009F00050F4877091E001C0990F8A95EAF7892F2A
:100A00000E94390DD9CF9BE5980F933020F480E0F8
:100A100090E00C94982598E5980F973120F480E0A9
:100A200090E00C94AE258D3E20F00E94F3160C94BD
:100A30006A1708951F93CF93DF93182FEB010E943D
:100A40000304209741F08FE99FE00197F1F700C080
:100A500000002197F6CF812FDF91CF911F910C9449
:100A6000B204893319F060E070E002C060E570E024
:100A70000C941A05882321F00E94330D0C94720DFA
:100A80000895882321F00E94390D0C94720D089569
:100A9000CF92DF92EF92FF920F931F93CF93DF934A
:100AA0007C01D62FC72FFC011281058102950F70A2
:100AB0000E94290D8823B9F01123A9F08C2F807F83
:100AC000803421F080E28D0F883068F08091D1026F
:100AD00082FD09C082E00E94D20D0E94290D91E0A2
:100AE000D82ED92601C0D12CCC2EC2948FE0C8229A
:100AF0008C2D90E08C30910508F0CFC1FC01EA5AB2
:100B0000FF4F0C945C2E8C2F807FCF70882311F0C8
:100B1000C295C07F112399F0CC2309F4AAC180E2C9
:100B20008D0F883010F0D11104C08C2F0E94330D2E
:100B300003C08C2F0E94430D0E94720D9AC18D2F0D
:100B40000E94B204CC2309F4A8C180E28D0F883042
:100B500038F1DD2329F18C2F0E94490D24C08C2F00
:100B6000807FCF70803211F0C295C07FDD2319F0F5
:100B7000D130A1F13DC08091D10282FF17C0112375
:100B800049F0CC2329F08C2F0E94330D0E94720D66
:100B900080E070C180E00E94B204CC2309F47DC1E2
:100BA0008C2F0E94390D0E94720D77C1112371F0B4
:100BB000002341F0013031F40E94530D8C2B0E9430
:100BC0005B0D6BC10E94530D8C2B1DC0002319F0CF
:100BD000013009F462C10E94680D25C0112321F083
:100BE000063008F05AC10EC0053008F056C11BC0CF
:100BF000112361F0002331F0F701858180FF39C1B5
:100C00008F7085838C2F0E943A0547C1002359F0CD
:100C1000D93309F03FC1FFEF07EE13E0F150004078
:100C20001040E1F735C18C2F0E94410536C18C2F51
:100C300086958695837019F0813061F02EC111235D
:100C400021F08D2F9C2F937002C080E090E00E94D5
:100C500098252BC1112321F08D2F9C2F937002C05A
:100C600080E090E00E94AE2520C18D2F112319F065
:100C70000E94981602C00E94F3160E946A1715C1BE
:100C80008C2F837009F047C011110BC12D2F2295B5
:100C900026952770220F220F6D2F6F70862F90E000
:100CA000A0E0B0E0022E04C0880F991FAA1FBB1F4E
:100CB0000A94D2F7D4FF10C04FE050E060E070E03B
:100CC00004C0440F551F661F771F2A95D2F7409521
:100CD00050956095709503C040E050E0BA01C6950C
:100CE000C695C3708A019B01082B192B2A2B3B2B1D
:100CF000C901B801C23049F058F4C13019F00E945E
:100D00004908CFC00E943708CCC00E945B08C9C008
:100D10000E943508C6C0112319F08C2F817001C0C4
:100D20008695882309F4BDC02D2F2295269527701E
:100D3000220F220F6D2F6F70862F90E0A0E0B0E0A1
:100D4000022E04C0880F991FAA1FBB1F0A94D2F756
:100D5000D4FF10C04FE050E060E070E004C0440FEA
:100D6000551F661F771F2A95D2F7409550956095BD
:100D7000709503C040E050E0BA01C695C695C370B7
:100D80008A019B01082B192B2A2B3B2BC901B80187
:100D9000C23049F058F4C13019F00E940E0981C0E8
:100DA0000E94FC087EC00E9420097BC00E946F0840
:100DB00078C0CF70112339F08C2F0E9495088D2FA9
:100DC0000E943A056EC08D2F0E9441058C2F0E9413
:100DD000B60867C0D23F21F128F4D03F41F0D13F9F
:100DE000C1F043C0D33F19F1D43F79F03EC0112385
:100DF00041F0053008F051C08C2F8F710E94DB0844
:100E00004CC0063008F049C0F7CF8091D10282FF74
:100E100018C0112339F08C2F8F710E9495083DC0A6
:100E20001123C9F38C2F8F710E94B60836C011238D
:100E300029F08C2F8F710E9480082FC00E947B08A0
:100E40002CC0112349F0CF718C2F0E94950863E0CC
:100E50008C2F0E94B70D21C081E00E94D20D02307C
:100E6000E0F082E00E94D20D18C0112331F000237F
:100E700091F28D2F0E94030410C0002399F2D93300
:100E800049F41FEF27EE33E0115020403040E1F7E6
:100E900000C000008D2F0E94B20488EF8C0D8430BA
:100EA00020F40E946C250E949803DD20C9F00E9466
:100EB000250D80FD15C0F70112820E941F0D0E94B2
:100EC0009508C7010E9491070E941F0DDF91CF91E5
:100ED0001F910F91FF90EF90DF90CF900C94B60888
:100EE000DF91CF911F910F91FF90EF90DF90CF9006
:100EF00008950F931F93CF93DF93EC01688179815D
:100F00008A810E94D7098C010E9432090E9423081D
:100F1000B801CE010E944805DF91CF911F910F913A
:100F20000895CF93DF93EC01988189812B813C81D7
:100F3000232B31F08F3F31F481E09F3F19F403C040
:100F400081E001C080E080FD1DC0CE010E942F0322
:100F5000811110C00E94290D8823A1F08A81882365
:100F600089F08091D10282FD0DC082E0DF91CF91A6
:100F70000C94D20DCE010E947907CE01DF91CF9162
:100F80000C941003DF91CF91089580E090E00E94CF
:100F9000982580E090E00E94AE250E94500D0E94AE
:100FA000720D0E949B180C946A1780910201909117
:100FB00003010E940A260C94C5070E94400D0C9460
:100FC000D50792959F70963079F010F4925001C039
:100FD0009A50923068F4803F69F018F4883E40F4EB
:100FE00009C0843F29F406C0883E20F0813F11F0FB
:100FF00080E0089581E00895FC01808191810E9444
:10100000CC090E94E1070895CF93DF9300D000D070
:101010001F92CDB7DEB70F900F900F900F900F90EB
:10102000DF91CF910895CF93DF9300D000D000D00F
:10103000CDB7DEB726960FB6F894DEBF0FBECDBF94
:10104000DF91CF910895089508950C9424080C948D
:1010500025080E94270860930D0270930E0280936A
:101060000F02909310020C94C5070C9429080F935B
:101070001F9300910D0210910E0220910F023091EA
:101080001002602B712B822B932B1F910F910C94CC
:1010900029080F931F9300910D0210910E022091C9
:1010A0000F023091100260237123822393231F913A
:1010B0000F910C9429080F931F9300910D0210912A
:1010C0000E0220910F0230911002602771278227B3
:1010D00093271F910F910C9429080C9424080E94C7
:1010E0006D086093090270930A0280930B0290933B
:1010F0000C020C94C50760E070E0CB010C946F0803
:101100000F931F9341E050E060E070E08A019B0183
:1011100004C0000F111F221F331F8A95D2F7C90187
:10112000B8011F910F910C946F080F931F9341E02A
:1011300050E060E070E004C0440F551F661F771F49
:101140008A95D2F78091090290910A02A0910B0230
:10115000B0910C028A019B01082B192B2A2B3B2BE7
:10116000C901B8011F910F910C946F080F931F9341
:1011700041E050E060E070E004C0440F551F661F7E
:10118000771F8A95D2F7409550956095709580911C
:10119000090290910A02A0910B02B0910C028A01FF
:1011A0009B01082319232A233B23C901B8011F915E
:1011B0000F910C946F080F931F9341E050E060E093
:1011C00070E004C0440F551F661F771F8A95D2F741
:1011D0008091090290910A02A0910B02B0910C0239
:1011E0008A019B01082719272A273B27C901B80133
:1011F0001F910F910C946F080F931F930091090298
:1012000010910A0220910B0230910C02602B712B7D
:10121000822B932B1F910F910C946F080F931F93A8
:101220000091090210910A0220910B0230910C02E8
:1012300060237123822393231F910F910C946F08D5
:101240000F931F930091090210910A0220910B0243
:1012500030910C0260277127822793271F910F91ED
:101260000C946F08089527E0929F800D1124E82FB9
:10127000E695E695E695877051E001C0550F8A9591
:10128000EAF785E0E89FF0011124E452FE4F20E0E8
:1012900030E070E04081CB01022E02C09695879528
:1012A0000A94E2F7817081958427852384278193AE
:1012B0002F5F3F4F2530310569F7089527E0929F52
:1012C000800D1124682F669566956695982F977006
:1012D00085E0689FB001112440E050E080E0FB0110
:1012E000E40FF51FE452FE4F208130E0092E02C0CA
:1012F000369527950A94E2F721703327042E01C012
:10130000220F0A94EAF7822B4F5F5F4F4530510559
:1013100031F70895BF92CF92DF92EF92FF920F9331
:101320001F93CF93DF938C01C0900902D0900A02E3
:10133000E0900B02F0900C0280910D0290910E0251
:10134000A0910F02B0911002C82AD92AEA2AFB2ADA
:10135000CFE1D0E0D701C6010C2E04C0B695A79509
:10136000979587950A94D2F780FD04C0219790F74E
:10137000B12C07C0BC2EB8018C2F0E94C41001975D
:10138000A9F38B2DDF91CF911F910F91FF90EF90DB
:10139000DF90CF90BF900895CF93DF93EC010E9430
:1013A0008A09BE010E94C410DF91CF9108951F9356
:1013B000CF93DF93EB019091DB01992321F0CB01D7
:1013C0000E94CC0913C0882349F0CB010E948A09EE
:1013D000182F682FCE010E94330904C0CB010E9450
:1013E0005E09182FBE01812F0E94C410DF91CF919A
:1013F0001F9108951F93CF93DF93C091110216E0C0
:1014000080911202C81799F0D0E01C9FF0011D9F37
:10141000F00D1124ED5EFD4F408151816281738199
:10142000848195810E9413082196C770E9CFDF91CE
:10143000CF911F91089540914302509144026091D1
:1014400045027091460280914702909148020C94A7
:101450001308EF92FF920F931F93CF93DF93809126
:10146000480282958F7009F065C0809145028823FB
:1014700009F460C080911102F090120210914302B1
:1014800000914402609146027091470291E01F3F33
:1014900009F090E0C0910001D0910101292F96E060
:1014A000E92E8F1509F446C06115710521F00F3F33
:1014B00021F030E003C031E001C0322F90E030FD78
:1014C00036C0E89EF001E99EF00D1124DF01AD5E0B
:1014D000BD4F11963C911197301329C03C913113A7
:1014E00026C012963C911297311121C013964D914E
:1014F0005C911497461B570B4C175D07C0F4809105
:1015000048028F70806180934802E85EFD4F8081C1
:101510008F708061808383E492E00E949107DF9165
:10152000CF911F910F91FF90EF900C94FA090196C3
:101530008770B7CFDF91CF911F910F91FF90EF9000
:1015400008959F92AF92BF92CF92DF92EF92FF9257
:101550000F931F93CF93DF93CDB7DEB761970FB68D
:10156000F894DEBF0FBECDBF8C0185E0F801DE012F
:101570001D9601900D928A95E1F7D8011296EC9094
:1015800090914302E091440220914602309147023B
:101590002115310531F0EF3F31F481E09F3F19F41F
:1015A00003C081E001C080E0B82FB1709B2E80FDA8
:1015B00047C1D8014C9111965C9111971396AD904B
:1015C000BC90149783E4C82E82E0D82EF090450298
:1015D000B501621B730B2091000130910101FF20C6
:1015E00009F4D9C0809148026217730708F095C0CA
:1015F000282F207F09F052C05E1313C0491311C079
:10160000FE2CE1100EC08F708061809348020E9412
:101610001B0AC6010E94910780914802F801858348
:101620004DC1AB2831F05F3F31F481E04F3F19F4F9
:1016300003C081E001C080E080FD03C081E08E2511
:1016400002C080E090E0F82FF170FF2E80FF1CC0F8
:10165000809111022091120236E0821709F40BC129
:1016600090E0389FF001399FF00D1124ED5EFD4FA1
:101670006181561306C06081461303C06281E61281
:1016800003C001968770E9CFFE2CEE2009F416C145
:101690008091480281608093480254C05E1306C066
:1016A000491304C0E11002C0F80199C0C8010E94AA
:1016B000FC07882361F1EE2051F120914802822F2E
:1016C00082958F7090E0029774F080914302909120
:1016D000440298878F831986BB86AA862C87CE0101
:1016E00007960E94910786E0F801A3E4B2E001901A
:1016F0000D928A95E1F70E94290A0E941B0A0AC0EE
:101700005E1711F1C8010E94FC0781112CC0C801AD
:101710000E949107FF24F394D1C0282F207F81F7E6
:101720007A2DB98AA88A6E2D89890E94040883E4DB
:1017300092E00E94910786E0D6011D928A95E9F712
:101740000E941B0AF12CBAC04913DCCFE110DACF9A
:10175000F8018583C8010E94910786E0D6011D9299
:101760008A95E9F7ABC0EE2091F220914802822FD2
:1017700082958F7090E002970CF4B5CF8091430270
:10178000909144029A8389831B82BD82AC822E830E
:10179000CE010196A6CF6217730708F044C0FE2C55
:1017A000EE2009F4B4CF5E1330C049132EC020914F
:1017B000480220FD21C0822F82958F70482F50E073
:1017C00041155105C9F0F80125834F30510541F00D
:1017D0008F5F982F9295907F822F8F70892B8583B2
:1017E000C8010E94910786E0F801A3E4B2E00190ED
:1017F0000D928A95E1F73CC086E0F801A3E4B2E0DF
:1018000001900D928A95E1F759C0C8010E94FC072A
:10181000811169CF80914802816080934802C8019C
:101820000E9491074BC07A2DB98AA88A6E2D8989AA
:101830000E94040886E0D6011D928A95E9F718C037
:10184000EE2009F464CFC8010E94FC07F82E88231B
:1018500009F45DCF86E0F801A3E4B2E001900D92B7
:101860008A95E1F783E492E00E94FD030E94290A31
:101870000E941B0A23C04D875E878D859E850E942E
:10188000CC09292F22952F70223028F49F7039F02F
:10189000811105C00BC0243028F49F7049F4805E8C
:1018A000883020F0C8010E9491079F2CF92C06C0B7
:1018B000D80115969C91907F91F7F8CF8F2D619666
:1018C0000FB6F894DEBF0FBECDBFDF91CF911F9151
:1018D0000F91FF90EF90DF90CF90BF90AF909F90CF
:1018E00008951F93CF93DF93CDB7DEB72C970FB634
:1018F000F894DEBF0FBECDBF4F83588769877A87C4
:101900008B879C87CE0107960E94A10A8823D1F07D
:101910009F8188852A853B85232B31F08F3F31F4C9
:1019200081E09F3F19F403C081E001C080E080FDA9
:1019300047C04F81588569857A858B859C850E9433
:1019400013083EC086E0FE013796DE011196019035
:101950000D928A95E1F7FF81E8856A857B8561159F
:10196000710531F0EF3F31F481E0FF3F19F403C01E
:1019700081E001C080E080FD23C02091120230E0B0
:10198000C9010196877099274091110250E0841790
:101990009507F1F1F983EA837D836C8396E0929F4A
:1019A000D001939FB00D1124AD5EBD4FFE01319665
:1019B00001900D929A95E1F7809312020E94FA0924
:1019C00016E08091110290911202891771F1189F0F
:1019D000C00111248D5E9D4F0E94A10A882329F128
:1019E000E09111021E9FF0011124ED5EFD4F408138
:1019F000518162817381848195810E941308809155
:101A0000110290E001968770992780931102D9CF37
:101A10000E94DD071092120210921102E3E4F2E03C
:101A200086E0DF011D928A95E9F72C960FB6F894AF
:101A3000DEBF0FBECDBFDF91CF911F910895809182
:101A400051028595859585950895809151028770FD
:101A5000089590915102977081E009F480E0089513
:101A600080915C02089590915C02892B80935C02C6
:101A70000895809590915C02892380935C0208957B
:101A800010925C02089590915B02892B80935B0217
:101A90000895809590915B02892380935B0208955D
:101AA00010925B02089580915202089508950C945B
:101AB000560D0C94570D9091D10292FD08C0909153
:101AC0005202981721F0809352020C94590D0895F8
:101AD00080915202882329F01092520280E00C94E7
:101AE000590D0895CF93DF93E0910201F091030126
:101AF00080915C028083E0910201F091030190816A
:101B000080915B02892B808380915202882381F02F
:101B1000E0910201F09103019081892B80838091F3
:101B20000201909103010E94C42581110E94680D59
:101B3000C0910201D091030148E050E069E472E0F5
:101B4000CE010E94AC2E892B69F088E0FE01A9E449
:101B5000B2E001900D928A95E1F7CE01DF91CF912D
:101B60000C947F25DF91CF9108950C94560D9091A0
:101B7000D10292FD10C098E0899F90011124262B7C
:101B8000209351020E949508809151028595859578
:101B900085950C94B50D0C9495081092510280E037
:101BA0000C94B50D209151028095822380935102AF
:101BB000982F977099F430E0482F082E000C550BA1
:101BC0002417350759F09091D10292FD07C08595F1
:101BD000859585950E94B6080C94CD0D0895909139
:101BE000D10292FB222720F9281769F080FB92F995
:101BF0009093D1028091D0029091D1020E94370E31
:101C000082E00C94D20D08958091D10282FB882746
:101C100080F991E089270C94EF0D81E00C94EF0D91
:101C200080E00C94EF0D80E090E00E94D02E21E047
:101C3000893E9E4F09F020E0822F089582E090E0D7
:101C40000C94C22E83E090E00C94C22ECF9384E0DB
:101C500090E00E94C22EC82F82E290E00E94C22E25
:101C60002C2F30E0A901582BCA01CF910895CF93B2
:101C7000C92F682F84E090E00E94D62E6C2F82E25C
:101C800090E0CF910C94D62EAB01BC018FE090E098
:101C90000C94E82EAB01BC0183E190E00C94E82E9B
:101CA00060E070E0CB010C944A0E60E070E0CB0184
:101CB0000E94440E0C94500E69EE7EEF80E090E09E
:101CC0000E94F42E60E082E090E00E94D62E60E058
:101CD00083E090E00E94D62E10920D0210920E0228
:101CE00010920F021092100260E084E090E00E94D7
:101CF000D62E60E082E290E00E94D62E60E085E081
:101D000090E00E94D62E60E086E090E00E94D62E01
:101D10006FEF87E090E00E94D62E40E050E0BA01DD
:101D200088E090E00E94E82E60E08DE090E00E9464
:101D3000D62E40E050E0BA0188E190E00E94E82E03
:101D400060E087E190E00E94D62E40E050E0BA01CA
:101D50008CE190E00E94E82E60E070E080E290E08C
:101D60000E94F42E40E050E0BA0188E190E00E9429
:101D7000E82E0C94550E0C945C0E682F8EE090E0CB
:101D80000C94D62E0E94B82660936B0270936C025E
:101D900080936D0290936E02609367027093680265
:101DA0008093690290936A02089585B7806885BF21
:101DB00085B7806885BF08950C94DB1308950C9453
:101DC000DE0E0C94DE0E0C94E10E0C94DE0E0C94E0
:101DD000E50E0C94DE0E0E94D50E8AEE91E10E9473
:101DE00062250E94E90E0C94E70E0E94DF0E0C940F
:101DF000DE0E0E94ED110C9497030E94A3260E9410
:101E0000A0110E94F5130E942C130E94F90E0E944B
:101E1000D51F0E94FA1D0E94FF130C94E30E8F92AF
:101E20009F92AF92BF92CF92DF92EF92FF920F9369
:101E30001F93CF93DF93CDB7DEB72A970FB6F894F1
:101E4000DEBF0FBECDBF0E945013982E81110E949D
:101E5000C20E8DE5A82E82E0B82E00E010E0802EA4
:101E6000802F0E941112D82EF501C1905F01C82663
:101E7000B1F40F5F1F4F0A30110589F78FEF898387
:101E80008A831B820E94AC268160782F9D838C837D
:101E900049815A816B818D810E94B3032FC080914B
:101EA0006F0281FD0E941712E12CFF24F3948C2D08
:101EB0008F21F1F00E94DC0E882399F0EE828F8250
:101EC000DF2081E009F480E088870E94AC268160F1
:101ED000782F9A8789874E815F8168858A850E94DD
:101EE000B303F801E35AFD4F8081F826F08206C063
:101EF000E394FF0CF7E0EF12DACFBBCF81E0911053
:101F000001C080E02A960FB6F894DEBF0FBECDBFA9
:101F1000DF91CF911F910F91FF90EF90DF90CF90C5
:101F2000BF90AF909F908F9008950E940F0F0E94D6
:101F3000DB130E942D1E0E9488170C94A803CF93D8
:101F4000DF930E94C910EC01811521E5920708F08A
:101F500045C0811530E5930708F094C0883E91058F
:101F600028F5803E910508F0F8C0883A910570F494
:101F7000853A910508F07CC08130910509F475C05F
:101F800008F4E8C0049708F0E8C0E4C08F3B91056E
:101F900008F0E0C0C85AD0E0CC0FDD1FCC58DE4FAF
:101FA0000990D881C02DCE019464D8C0811540E23B
:101FB000940758F4811551E0950708F0CEC08D3E86
:101FC000910508F4C7C09065C9C0C11580E4D80761
:101FD00008F4C0C0DF70CE01906AC0C0811525E54D
:101FE0009207A8F4811534E5930708F095C0811590
:101FF00043E5940708F07BC0811552E5950708F08A
:1020000061C0D82FCC27CE01816F906AA7C0C115BF
:1020100089E5D807A0F4C11528E5D20708F082C0E9
:10202000C11536E5D30708F095C08C2F0E945D11CD
:102030008F7190E0D82FCC27CE0190628FC0C11550
:102040004AE5D40708F474C0CE0190568115904239
:1020500008F080C08D2F8F710E945D11DD27D06246
:102060008F71AE01582BCA0179C081E090E076C033
:10207000C55AD0E0CE55DE4F8881C82FD0E0CE01C2
:1020800090646CC074E0969587957A95E1F7282F57
:1020900023703C2F337081E090E002C0880F991FBD
:1020A0003A95E2F79C68AC01522B9A019C2F9F70E5
:1020B0009695969550E2959FE0011124C9018C2BCD
:1020C0009D2B4CC08370992721E030E002C0220F85
:1020D000331F8A95E2F79C2F9695969580E2989FFC
:1020E000E0011124C22BD32BCE019C6837C0837032
:1020F000992721E030E002C0220F331F8A95E2F7D2
:102100009C2F9695969540E2949FE0011124C22B56
:10211000D32BCE019A6822C0D82FCC27CE01846F52
:10212000906A1CC0DC2FCC27CE01806F906A16C04D
:102130008C2F8F700E945D1194E0D695C7959A956B
:10214000E1F7CF70D0E0DC2FCC27D0699E01282B9F
:10215000C90104C080E090E001C0CE01DF91CF91C1
:10216000089526E4829FC0011124FC0127E0729F9C
:10217000E00DF11D1124E60FF11DEE0FFF1FE852D7
:10218000FF4F8591949108950E94B1100E949F0F76
:1021900008958238910569F1B0F48133910509F40D
:1021A0006DC048F48932910509F463C08A32910503
:1021B00009F469C008958533910509F455C0893340
:1021C0009105B9F00895833E910569F138F4803E98
:1021D0009105B1F0823E910509F10895863E910581
:1021E000A9F1873E9105B9F1843E910509F064C0DB
:1021F00023C02091D00220FD4FC021FD4DC0089585
:102200008091D00280FD44C08091D10280FF44C003
:102210008091D00284FD42C083EE4DC08091D002F7
:1022200082FF38C0F5CF8091D00282FD33C080910B
:10223000D10280FD31C0ECCF8091D10281FF32C04C
:102240008091D00284FD2AC087EE35C08091D002F3
:1022500083FF26C0F5CF8091D00283FD21C08091FD
:10226000D10281FD1FC0ECCF8091D00285FD1CC042
:102270001DC08091D00285FD19C016C08091D0028A
:1022800086FD16C017C08091D00286FD13C010C015
:1022900089E311C082EE0FC080EE0DC080E00BC05C
:1022A00086EE09C084EE07C089E205C085E303C05D
:1022B0008AE201C081E390E008959091D00292FFFC
:1022C0000DC0282F2871283019F4877F846006C03C
:1022D000282F2471243011F48B7F886093FF0DC068
:1022E000282F2871283119F4877E846106C0282F91
:1022F0002471243111F48B7E88612091D10220FF5A
:102300000DC0382F3871383019F4877F816006C0CE
:10231000382F3171313011F48E7F886021FF0DC06C
:10232000282F2871283119F4877E816106C0282F53
:102330002171213111F48E7E886194FD877E08958C
:102340001092CC021092CD021092CE021092CF02C7
:102350000895CF92DF92EF92FF926B017C010E9471
:10236000DB1381110EC00E94B826C61AD70AE80AEC
:10237000F90AC092CC02D092CD02E092CE02F09245
:10238000CF02FF90EF90DF90CF9008950F931F93AF
:102390000E94DB13882321F01F910F910C94B82623
:1023A0000E94B8260091CC021091CD022091CE025D
:1023B0003091CF02600F711F821F931F1F910F91E9
:1023C00008950E94DB1381110C94AC260E94C61163
:1023D000CB01089580E0089508950E94130E8111A5
:1023E00002C00E94BB0E0E941E0E80936F020E94CC
:1023F000260E9093D1028093D0020E94EC110E948D
:10240000220E682F70E080E090E00E943508609115
:10241000090270910A0280910B0290910C020C94B7
:102420006D08E82FF0E0E352FD4F80810895089594
:1024300080EA8A95F1F7089500C008950C94181267
:1024400008950C9420120C9421120C9420120C94D8
:1024500025120C942012FF920F931F93CF93DF93BA
:1024600000D000D01F92CDB7DEB70E94DB13609181
:10247000E7028823E9F185E0F82E8E010F5F1F4FF8
:10248000F8018F2D11928A95E9F7862F90E0B80117
:1024900083529D4F0E940D14882389F08091D202AF
:1024A00090E045E050E0B80183529D4F0E94AC2E71
:1024B00021E020937002892B61F410E016C0809116
:1024C00070028823D1F3F8011192FA94E9F710927F
:1024D0007002A091D202B0E0A352BD4F85E0F80196
:1024E00001900D928A95E1F711E00E941D030DC045
:1024F00070E063527D4F8091D20290E083529D4FF5
:102500000E9497140E94291210E0812F0F900F90C3
:102510000F900F900F90DF91CF911F910F91FF902F
:102520000895F894E82FE295EF70F0E031A1282F9C
:102530002F7081E090E001C0880F2A95EAF7982F6C
:102540009095932391A392A1892B82A378940895C7
:102550000F931F93CF93DF93CCEAD1E089918F3F04
:1025600011F00E94911281E0C13BD807B9F7C5EA8A
:10257000D1E00CEA11E089918F3F11F00E94911295
:102580000C171D07C1F7DF91CF911F910F9108958F
:10259000CF92DF92EF92FF920F931F93CF93DF932F
:1025A0008C01C62FD0E0CE0184559E4F7C01FC01EA
:1025B00090819F3F09F447C0D62EF894E92FE29509
:1025C000EF70F0E081A19F7021E030E001C0220FA8
:1025D0009A95EAF7822B81A382A12095282322A332
:1025E00078940E941C12E5EAF1E04CEA51E031E0F7
:1025F000C12C21912F3F89F0A22FA295AF70B0E09E
:1026000090968C9190E02F7002C0959587952A95B1
:10261000E2F780FD02C0832F01C080E0C82A330F9B
:102620004E175F0731F7F70180818F3F11F00E944D
:10263000911261E0C11001C060E08D2D0E941E1258
:10264000C00FD11FC882DF91CF911F910F91FF90D2
:10265000EF90DF90CF900895809104018091040164
:10266000811102C095E001C090E09093E70285E0FF
:10267000891B8093D2020E94A8128AE0EDEDF2E05D
:10268000DF01982F1D929A95E9F7E3EDF2E0DF0163
:102690001D928A95E9F785E00E94A4130C941B0310
:1026A000EF92FF920F931F93CF93DF93CDB7DEB7D7
:1026B0002A970FB6F894DEBF0FBECDBF8E010F5F15
:1026C0001F4F8AE0F80111928A95E9F7F12C6F2DDE
:1026D000C8010E94C812F394F5E0FF12F8CF4AE057
:1026E00050E0B80183ED92E00E94AC2E7C0121E025
:1026F000892B09F420E0E114F10441F08AE0F801AB
:10270000A3EDB2E001900D928A95E1F76091E702A6
:1027100070E063527D4F45E083ED92E00E94A51387
:10272000EF2819F40E942B1202C081E090E02A9653
:102730000FB6F894DEBF0FBECDBFDF91CF911F91D2
:102740000F91FF90EF9008950895FF920F931F93BC
:10275000CF93DF938C01F62ED72FC42F222349F07D
:1027600081E0809373020E94AC2690937202809362
:102770007102809173028823C1F08091710290915F
:1027800072020E94C426059780F0EF2DFD2FD8011C
:102790004C2F50E0CD01801B910B841795071CF442
:1027A0008D918193F7CF10927302DF91CF911F919A
:1027B0000F91FF9008958091760281110DC00E94C3
:1027C000F72D811102C082E001C081E08093760282
:1027D000823011F40E94F22D81E0909176029130C6
:1027E00009F080E008950C94DB130E94F3138093AA
:1027F00004010E94DB1381110C94451408950E947A
:10280000DB13811102C00C944714089581E090916C
:1028100077029A3008F080E008950F931F93CF93CA
:10282000DF93EC018B01809177028A3038F4B80194
:10283000CE010E94951481111DC00AC080917402BE
:10284000909175020E94C426843F914080F715C084
:10285000809177028F3F19F08F5F8093770280918C
:1028600077028A3060F00E94AC26909375028093C4
:10287000740203C01092770202C080E001C081E0C0
:10288000DF91CF911F910F9108950C94FB230C942D
:10289000FE23DF92EF92FF920F931F93CF93DF936C
:1028A0007901C82F880FDD0B41155105A9F0FE01F4
:1028B00093E0EE0FFF1F9A95E1F7EB5FFE4F8181EA
:1028C000928188589D4F208130E04217530708F4C9
:1028D0009A01A9010E94B92ECE010E94E724D82EA8
:1028E0008823D1F001151105B9F083E0CC0FDD1F6D
:1028F0008A95E1F7FE01EB5FFE4F438150E004173C
:10290000150708F4A801CB5FDE4F6C817D81685804
:102910007D4FC7010E94B92E8D2DDF91CF911F9160
:102920000F91FF90EF90DF9008950C94B1150C94E7
:10293000CD150F931F93CF93DF9300D000D0CDB769
:10294000DEB760918F027091900280919102909118
:1029500092020E94D326643671058105910528F103
:102960000E94C611DC01CB010296A11DB11D898315
:102970009A83AB83BC8300E010E020E030E044E0C9
:1029800050E0BE016F5F7F4F82E00E944914182F14
:10299000882361F00E94B82660938F0270939002A2
:1029A000809391029093920201C011E0812F0F90C9
:1029B0000F900F900F90DF91CF911F910F9108957D
:1029C000AF92BF92CF92DF92EF92FF920F931F933D
:1029D000CF93DF937C015B016A010E940614811191
:1029E00003C001E010E002C00AE010E0C1E0D0E066
:1029F000F894B501C701F60109957894811115C0C5
:102A000021960C171D0794F0CC9F9001CD9F300D9F
:102A1000300D112480E090E045E34A95F1F7000085
:102A2000019682179307C1F7E3CF81E0DF91CF9141
:102A30001F910F91FF90EF90DF90CF90BF90AF90DC
:102A40000895AF92BF92CF92DF92EF92FF920F93D1
:102A50001F93CF93DF9300D000D000D0CDB7DEB767
:102A60007B01C090B101D090B20101E010E09E0165
:102A70002A5F3F4F40E050E060E070E080E00E945D
:102A80004914182F882309F43EC056018FEFA81A65
:102A9000B80A60918B0270918C0280918D029091A6
:102AA0008E020E94D326643671058105910518F1C6
:102AB00005E010E09E012F5F3F4F40E050E060E0F6
:102AC00070E081E00E944914182F65E070E0C501B4
:102AD0000E94D61F91E02E81281390E0192339F12E
:102AE0000E94B82660938B0270938C0280938D02B3
:102AF00090938E0211C065E070E0C5010E94D61F60
:102B00009E818913D5CF85E0F6013196DE011196BD
:102B100001900D928A95E1F7112349F085E0FE01BD
:102B20003196A6E8B2E001900D928A95E1F785E032
:102B3000E6E8F2E0D70101900D928A95E1F7812F46
:102B400026960FB6F894DEBF0FBECDBFDF91CF91B2
:102B50001F910F91FF90EF90DF90CF90BF90AF90BB
:102B600008950F931F93CF93DF93EC018B0141E204
:102B700055E10E94E014882351F049E954E1B8017D
:102B8000CE01DF91CF911F910F910C94E01480E062
:102B9000DF91CF911F910F9108950F931F93CF93C2
:102BA000DF93F894C091B101D091B201CE010196AA
:102BB00025E0FB01DC0101900D922A95E1F765E02B
:102BC00070E00E94D61F88837894F8946E817F818C
:102BD0008885998500918202109183022091840258
:102BE00030918502601771078207930751F0609357
:102BF00082027093830280938402909385020E94E4
:102C0000A9117894DF91CF911F910F9108950E949F
:102C1000B8280E94FD0E0C94C4280E94C8280E9467
:102C2000950F0C94E2280E944A260E949F280E9439
:102C3000EB0E0E9407160E940D160E94F50EFBCFA8
:102C400080919B0280FF06C06091210170E0660FB9
:102C5000771F26C081FF04C06091210184E005C078
:102C600082FF07C06091210188E0689FB0011124B4
:102C700017C090919A029923D1F060912001961784
:102C800088F72091210188E0289F90011124929FCC
:102C9000A001939F500D112470E0CA010E94262EBE
:102CA0006038710540F46115710519F406C068E0DB
:102CB00070E0862F08958FE7089581E00895809150
:102CC0009B0280FF08C060911E0170E075956795BA
:102CD0007595679521C081FF06C060911E0170E067
:102CE0007595679519C082FF04C060911E0170E060
:102CF00010C090919902992399F060911D01961747
:102D0000A0F780911E01899FC001112470E00E94EC
:102D1000262E6038710540F46115710519F406C05E
:102D200061E070E0862F08958FE7089581E00895AF
:102D30008D3E21F40E942016819504C08E3E29F418
:102D40000E94201680939F0208958F3E21F40E94D6
:102D50002016819504C0803F29F40E94201680939C
:102D60009E020895893F19F40E945F1605C08A3FAC
:102D700031F40E945F1681958093A00208958B3FE5
:102D800021F40E945F16819504C08C3F29F40E94B3
:102D90005F168093A10208959FE0980F983078F411
:102DA00021E030E0A90102C0440F551F9A95E2F7D7
:102DB000CA0190919D02892B80939D0208958D3FB9
:102DC00021F480919B0281600BC08E3F21F48091A1
:102DD0009B02826005C08F3F29F480919B02846032
:102DE00080939B0208958D3E39F490919F0297FF46
:102DF00035C010929F0259C08E3E29F490919F02D7
:102E00001916BCF32BC090919E028F3E29F497FFB8
:102E100025C010929E0249C0803F19F41916CCF3C8
:102E20001DC09091A002893F29F41916BCF410929C
:102E3000A0023BC08A3F19F497FF10C0F8CF8B3F28
:102E400039F49091A10297FF09C01092A1022DC000
:102E50008C3F21F49091A1021916BCF39FE0980FCA
:102E6000983080F421E030E0A90102C0440F551FE2
:102E70009A95E2F7CA01809590919D0289238093EB
:102E80009D0213C08D3F21F480919B028E7F0BC069
:102E90008E3F21F480919B028D7F05C08F3F29F4E6
:102EA00080919B028B7F80939B0280919E02811177
:102EB00006C080919F02811102C010929A028091F7
:102EC000A002811106C08091A102811102C010925E
:102ED000990208950E94AC2620919E02211104C0FF
:102EE00020919F02222321F09093980280939702D1
:102EF0002091A002211104C02091A102222321F0DF
:102F000090939602809395028CE992E00C948A2526
:102F1000EF92FF920F931F93CF93DF9300D000D0D7
:102F200000D0CDB7DEB786E0ECE9F2E0DE01119625
:102F300001900D928A95E1F7E0909E02F0909F0239
:102F40000091A0021091A10210929E0210929F0285
:102F50001092A0021092A102E11003C0FF2009F418
:102F60005DC080919702909198020E94C426AC01A6
:102F700090919A02992339F02091220130E0241790
:102F8000350758F04BC0209194028AE0289F9001A9
:102F900011242417350718F041C09F3F19F09F5F97
:102FA00090939A02EE2061F00E9420161E1414F0F5
:102FB0009FEF01C091E0989F902D112490939E0265
:102FC000FF2061F00E9420161F1414F09FEF01C033
:102FD00091E0989F902D112490939F0230919E0232
:102FE0003323E1F020919F022223C1F045EB34030B
:102FF000C0011124992319F090939E0203C081E02F
:1030000080939E0235EB2303C0011124992319F00C
:1030100090939F0203C081E080939F02011103C03F
:10302000112309F45DC080919502909196020E944F
:10303000C426AC0190919902992339F020911F0187
:1030400030E02417350758F04BC0209193028AE0F6
:10305000289F900111242417350718F041C09F3F85
:1030600019F09F5F90939902002361F00E945F1610
:10307000101614F09FEF01C091E0989F902D11243D
:103080009093A002112361F00E945F16111614F0B4
:103090009FEF01C091E0989F902D11249093A10281
:1030A0003091A0023323E1F02091A1022223C1F04C
:1030B00045EB3403C0011124992319F09093A00229
:1030C00003C081E08093A00235EB2303C0011124EB
:1030D000992319F09093A10203C081E08093A1028B
:1030E00080919E0281110BC080919F02811107C0C7
:1030F0008091A002811103C08091A10281110E94E0
:103100006A17EB82FC820D831E8386E0FE013196F6
:10311000ACE9B2E001900D928A95E1F726960FB6E0
:10312000F894DEBF0FBECDBFDF91CF911F910F91FD
:10313000FF90EF900895ECE9F2E086E0DF011D9248
:103140008A95E9F710929A021092990210929B02C6
:103150000895EF92FF920F931F93CF93DF938B010C
:10316000682F11110AC0442329F0E82FF0E0E95F2D
:10317000FC4F6491762F862F75C0212F30E0E82F09
:10318000F0E0442321F0E95FFC4FE491F0E046E0F9
:10319000049FC0011124CFEFD0E0BE010E94122E87
:1031A0004BEA4603C001479F900D1124800F911DEB
:1031B000800F911D982F990F890FAE01421B530B61
:1031C0004E9FD0014F9FB00D5E9FB00D11249B2FDD
:1031D000189FA0011124452F55278E01041B150BA4
:1031E0000E9FA0010F9F500D1E9F500D11247E01B8
:1031F000E81AF108E29E8001E39E100DF29E100D88
:103200001124212F3327C21BD30BCE9F9001CF9FB8
:10321000300DDE9F300D112462307105A9F048F4A5
:103220006115710569F061307105C9F48B2F752F37
:103230000DC06430710581F058F06630710579F485
:103240007E2F8B2F932F0DC0832F7B2F9E2F09C096
:103250008E2F7B2F952F05C08E2F732F02C07E2FB0
:10326000852F692FDF91CF911F910F91FF90EF90E4
:10327000089541E00E94A918089508950E943919FF
:103280000895CF93DF93762FE901682F842F0E9452
:103290003E19798368838A83DF91CF910895809165
:1032A000E802282F269530E02115310519F48170A8
:1032B000826005C02532310524F0817088648093D6
:1032C000E802089588E090E00C94CA2ECF92DF9235
:1032D000EF92FF926B017C010E944F19B701A6018A
:1032E00088E090E0FF90EF90DF90CF900C94E82E74
:1032F000E8EEF2E083E0808311828FEF82838383A4
:10330000148260817181828193810C94661980910D
:10331000E80280FF02C08695089580E008959091AC
:10332000EC02933018F49F5F9093EC02882351F0E5
:103330006091E8027091E9028091EA029091EB02BB
:103340000C946619089581E00C948F199091EC0209
:10335000992319F091509093EC02882351F06091D9
:10336000E8027091E9028091EA029091EB020C94DC
:103370006619089581E00C94A61970E00C94AA1FB8
:10338000609127018091E80280FF0AC080912601A8
:1033900023E0829FC001112483519D4F0C94BD19DD
:1033A0008091280190912901891780F7E82FF0E09A
:1033B0009F01220F331FE20FF31FE351FD4F1182D4
:1033C000108212828F5FF0CF9091E80290FF16C0BA
:1033D0009091280120912901921770F4E92FF0E0D3
:1033E000DF01AA0FBB1FEA0FFB1FE351FD4F8183D3
:1033F000608342839F5FF0CF0C94C0190895CF93F0
:10340000DF9300D01F92CDB7DEB79091E80290FF16
:103410000AC09E012F5F3F4F0E9441194B81698175
:103420008A810E94E4190F900F900F90DF91CF9145
:103430000895CF93DF93EC01EC81F0E0EE5FFD4F58
:103440004491E8EEF2E0628181810E94FF198C8153
:103450008F5F8C83DF91CF910895CF93DF93EC0141
:10346000E8EEF2E0438162818C810E94FF198C8139
:103470008F5F8C83DF91CF9108950F931F93CF932C
:10348000DF9300D01F92CDB7DEB78C018091A202EE
:1034900081110AC09E012F5F3F4F4FEF6FEF0E94D7
:1034A00041198A818093A202F8018481813051F010
:1034B00028F0823061F44091A2020AC08091A202F9
:1034C00040E007C06091A20240E080E003C040E01D
:1034D00080E060E00E94E419F801848190E00196A8
:1034E00063E070E00E94262E84830F900F900F906F
:1034F000DF91CF911F910F910895AF92BF92CF921C
:10350000DF92EF92FF920F931F93CF93DF9300D040
:103510001F92CDB7DEB7182FF62E042FE22E909112
:10352000E80290FF6DC0E92FE695AE2FB0E0AD54F4
:10353000BE4F8C918093AC029E7F923061F49E01CD
:103540002F5F3F4F812F0E9441194B8169818A81F2
:103550000E94E41943C0823019F40091EB023EC08E
:10356000863019F41091E90239C08930D9F38931D4
:10357000A9F5E9518E2F8170D82EE695F0E0EE5F27
:10358000FC4FA590B490C12CBB2460912A01C616B3
:1035900018F52C2D30E0A29EC001A39E900DB29E86
:1035A000900D112470E00E94122E812FD11002C0C4
:1035B000860F01C0861B90912801290F311DA9019A
:1035C000440F551F240F351F23513D4F402F6F2DA2
:1035D0000E944119C394D9CF0E94C0191093E902E7
:1035E000F092EA020093EB02EE2051F06091E802C3
:1035F0007091E9028091EA029091EB020E946619B3
:103600000F900F900F90DF91CF911F910F91FF902E
:10361000EF90DF90CF90BF90AF900895E8EEF2E08A
:103620009181282F4381628188E0890F0C947D1A53
:1036300081E00C940E1BE8EEF2E09181282F43818B
:10364000628188EF890F0C947D1A81E00C941B1B1A
:10365000E8EEF2E0628128E0620F08F46FEF282FB5
:10366000438181810C947D1A81E00C94281BE8EE43
:10367000F2E0628128E0621B08F460E0282F4381B9
:1036800081810C947D1A81E00C94371BE8EEF2E006
:10369000438128E0420F08F44FEF282F6281818197
:1036A0000C947D1A81E00C94461BE8EEF2E0438115
:1036B00028E0421B08F440E0282F628181810C94AD
:1036C0007D1A81E00C94551B20E00C947D1AFF922A
:1036D0000F931F93CF93DF93EC01F12C0FEF10E0CA
:1036E00060912A01F616F0F4809128012F2D30E028
:1036F000280F311DC901880F991F280F391F235129
:103700003D4F70E0C8010E94262E962F8C8140917B
:10371000EB026091EA02F99E800D11240E9441198A
:10372000F394DECF0E94C0199A818C8190FF02C071
:103730008F5F01C081508C83DF91CF911F910F91DA
:10374000FF900895AF92BF92CF92DF92EF92FF92D7
:103750000F931F93CF93DF93FC01828180FF02C000
:103760000FEF01C001E010E04EE0A42E80912A018D
:10377000181708F043C080912801C12ED12CE60112
:10378000C80FD11DCE01880F991FC80FD91FC35173
:10379000DD4F198218821A8234E0E32EF12CB12C0D
:1037A0008091A4028B0D8F302CF06A2D0E94042E84
:1037B000892F05C087FF03C090912A01890F082E29
:1037C000000C990BC816D90691F48091EB028E9DDE
:1037D000A0018F9D500D11245595479555954795FE
:1037E0009E016091EA028091E9020E944119B00EA7
:1037F000F1E0EF1AF108A1F61F5FB8CF0E94C019DF
:103800008091A402013031F4811102C080912A011B
:10381000815007C090E0019660912A0170E00E94FB
:10382000262E8093A402DF91CF911F910F91FF90DC
:10383000EF90DF90CF90BF90AF900895CF9380919D
:10384000280190912901891770F4E82FF0E09F0179
:10385000220F331FE20FF31FE351FD4F118210823D
:1038600012828F5FF0CFC0E060912A01C617C0F5C9
:10387000EC2FF0E070E0CF010E94262E209128016D
:10388000820F2091A302022E000C330B90E0E2176E
:10389000F307CCF020912501022E000C330B2E17DC
:1038A0003F078CF09C01220F331F820F931F9C0156
:1038B00023513D4F4091EB026091EA028091E90271
:1038C0000E9441190BC0FC01EE0FFF1F8E0F9F1FBE
:1038D000FC01E351FD4F118210821282CF5FC4CFF1
:1038E0000E94C019209124018091A302820F80932D
:1038F000A30290912501920F9093250119165CF473
:10390000082E000C990B40912A0150E041505109BA
:10391000841795071CF0219520932401CF910895D9
:103920008F929F92AF92BF92CF92DF92EF92FF92CF
:103930000F931F93CF93DF938C01FC014481C42F1D
:10394000D0E09E01DE010E946A2E9B01AC010E9424
:10395000802E6B017C01E0E2F0E0EC1BFD0BA5E5A5
:10396000B0E09B01AC010E94802E4B015C019F01E5
:10397000DF010E94622E9B01AC010E948B2E9B01F5
:10398000AC012C0D3D1D4E1D5F1DC501B4010E94F3
:103990003A2EC22FD22F2A3228F4F3E02F9F900123
:1039A00011240DC025E530E02C1B3109C901880F19
:1039B000991F280F391F37FF02C02F5F3F4F3595E2
:1039C0002795C22FC095F12C85E5E82EED1A809140
:1039D0002A01F816C8F4F1FC02C08E2D01C08D2F0B
:1039E000909128012F2D30E0290F311DA901440F9E
:1039F000551F240F351F23513D4F4C2F6091EA0274
:103A00000E944119F394E3CF0E94C019F801848108
:103A1000811102C091E003C0803219F49FEF9093AE
:103A2000230190912301890FF8018483DF91CF91C5
:103A30001F910F91FF90EF90DF90CF90BF90AF90CC
:103A40009F908F9008950F931F93CF93DF93EC0176
:103A500000E010E080912A01282F30E002171307C0
:103A600024F5909128019801290F311DA901440FD7
:103A7000551F240F351F23513D4F869590E04C81F3
:103A8000081719071CF4442331F002C0411103C088
:103A90004091EB0201C040E06091EA028091E902AE
:103AA0000E9441190F5F1F4FD5CF0E94C0198C8112
:103AB00090E00196817099278C83DF91CF911F91BF
:103AC0000F910895E8EEF2E080818E7F808360811F
:103AD0007181828193810E9466191092AD022FEF4D
:103AE00080E792E0215080409040E1F700C0000064
:103AF0000C94C0196091E802669570E04BE050E0CC
:103B00008BE291E00E949F2E892B19F481E0809333
:103B1000AD020E94E1119093A6028093A502089540
:103B20009091E80290FF35C09170811102C09260BF
:103B300006C0853210F0986402C0880F982B9093CD
:103B4000E802662351F06091E8027091E9028091E9
:103B5000EA029091EB020E9466196091E802669574
:103B600070E04BE050E08BE291E00E949F2E892BA9
:103B700019F01092AD0202C00E947A1D81E080937C
:103B8000A8024091EB026091EA028091E9020C9454
:103B9000641B0895682F9091E802969581E0890F43
:103BA000853208F081E00C94901D81E00C94CA1DD0
:103BB000682F9091E80296958FEF890F09F484E2BF
:103BC0000C94901D81E00C94D81D61E00C94901D24
:103BD000E8EEF2E080818160808386950C94E51D9B
:103BE0008091E80280FD0C94621D0C94E81D60E059
:103BF0000C94901D8091AB0281112EC00E94130E77
:103C0000811104C00E94BB0E0E9478190E946219A3
:103C10006093E8027093E9028093EA029093EB02CA
:103C20006E7F61F40E9478190E9462196093E80225
:103C30007093E9028093EA029093EB020E944F197D
:103C40001092AD028091E80280FF03C086950E9429
:103C5000F71D81E08093AB0208950F931F93CF93DC
:103C6000DF938091AD02882309F485C08091AC0276
:103C7000E091E802E695E81BE093A702823049F460
:103C8000F0E0E250FE4FE491CE2FD0E009E11AE1DE
:103C900049C0863049F4F0E0E550FE4FE491CE2F64
:103CA000D0E00DE21AE13EC0893051F4E695F0E033
:103CB000E850FE4FE491CE2FD0E007E61BE132C082
:103CC0008F3051F4E695F0E0EB50FE4FE491CE2FAB
:103CD000D0E002EA1BE126C0853149F4F0E0EE5065
:103CE000FE4FE491CE2FD0E00EE11CE11BC08831E5
:103CF00081F0833239F4E0EFF1E0C591D4910DE326
:103D00001AE110C0843251F4C4EFD1E003E21DE1A6
:103D100009C0C8E2D0E000E91CE104C0C0EDD7E072
:103D20000DE319E18091A802882361F01092A802A6
:103D30000E94E1119093A6028093A5021092AA021C
:103D40001092A9020E94E111E091A502F091A60251
:103D50008E1B9F0B8F3F9F4770F4EC0FFD1FF0935E
:103D6000A602E093A50285EA92E0F801DF91CF91E7
:103D70001F910F910994DF91CF911F910F91089599
:103D8000882311F0FA0101C0FB010994CF93DF935E
:103D9000C82FD62F0E9487198C1740F00E948719D0
:103DA0008D1720F4DF91CF910C94D51D8C2FDF91CE
:103DB000CF910C94E51D1F93CF93DF93FB011281EC
:103DC0001111C3C0EC010E94300D8272CD3CFCE5A4
:103DD000DF0709F49AC0A8F5C73CECE5DE0709F453
:103DE00076C0A8F4C43C9CE5D90709F45FC028F468
:103DF000C33CDC4509F457C054C0C53C9CE5D90719
:103E000009F459C0C63CDC4509F45CC04AC0CA3C50
:103E1000FCE5DF0709F46AC050F4C83CECE5DE07B6
:103E200009F45AC0C93CDC4509F45BC03AC0CB3C3C
:103E30009CE5D90709F45FC0CC3CDC4509F460C0BF
:103E400030C0C23DFCE5DF0709F46FC088F4CF3C09
:103E50009CE5D90709F460C008F45CC0C03DFCE5EE
:103E6000DF0709F45CC0C13DDC4509F45BC019C043
:103E7000C53D9CE5D90709F460C050F4C33DFCE59D
:103E8000DF0709F455C0C43DDC4509F454C009C03E
:103E9000C63D9CE5D90709F455C0CE35DD4509F48A
:103EA00054C011E052C00E94F01D4FC042EE5DE1CF
:103EB00065ED7DE104C045ED5DE162EE7DE10E94CE
:103EC000C01E43C045E25BE168E17BE1F8CF48E119
:103ED0005BE165E27BE1F3CF43E45BE164E37BE13B
:103EE000EECF44E35BE163E47BE1E9CF41E65BE1F4
:103EF00062E57BE1E4CF42E55BE161E67BE1DFCFB8
:103F00004AEB59E163EA79E1DACF43EA59E16AEB36
:103F100079E1D5CF81E017C065E082E010C068E0AC
:103F200086E00DC06EE089E00AC064E18FE007C062
:103F300067E185E104C088E106C062E289E10E9490
:103F4000C61E03C083E20E94E51D812FDF91CF9141
:103F50001F910895539A2BB1277F3BB138604FB71B
:103F6000F894FC01CB01880F991F680F791F6E0F21
:103F70007F1FE617F70789F0819198E03BB90000B1
:103F800000C087FF2BB9880F000000C000C000C030
:103F90002BB900C09A9591F7ECCF4FBF8FE594E015
:103FA0000197F1F700C0000008950895FC01680F23
:103FB000791F8FEF91E3E617F70771F021918227C0
:103FC00028E030E087FF03C0880F892701C0880FF1
:103FD00021503109B9F7EFCF0895CF93DF93EC016A
:103FE000FB018281882309F43CC1C430FDE5DF0771
:103FF00060F4CB3F9CE5D90788F49E0122503C45F4
:104000002431310508F02EC109C0C236EDE5DE07C6
:1040100029F0C63AFDE5DF0709F024C10E94260E0B
:104020009093D1028093D002C1318CE5D80709F476
:10403000C6C008F042C0C930ECE5DE0709F49BC0F9
:1040400000F5C5308CE5D80709F485C078F4C33095
:10405000ECE5DE0709F478C008F07AC0C230DC4530
:1040600009F0F5C08091D0028160EFC0C7309CE5B7
:10407000D90709F478C008F07AC08091D002806135
:10408000E4C0CD30FCE5DF0709F487C058F4CB303D
:104090009CE5D90709F479C008F07BC08091D00273
:1040A00088606FC0CF30FCE5DF0709F480C008F0FE
:1040B00082C08091D002877FC8C0CE3F9CE5D907DF
:1040C00009F471C000F5C531FCE5DF0709F485C0CE
:1040D00068F4C3319CE5D90709F475C008F095C0B0
:1040E0000E94DD078091D0028F77AFC0CC3FFCE506
:1040F000DF07A9F108F054C0CB3FDC4509F0A7C0A9
:104100008091D10240C0C230EDE5DE0709F489C0DC
:1041100058F4C1158DE5D80709F45AC008F069C0F4
:104120008091D10282602FC0C236EDE5DE0709F42E
:104130007CC0C63AFDE5DF0709F481C0C330DD4528
:1041400009F085C080E06EC08091D00282607DC0A1
:104150008091D00216C08091D002886076C0809194
:10416000D10282604FC08091D00280626EC0809187
:10417000D00280646AC00E94DD078091D00280680E
:1041800064C0846062C081603DC08091D0028E7F37
:104190005CC08091D0028D7F58C08091D00216C043
:1041A0008091D10218C08091D1028D7F2BC0809167
:1041B000D0028F7E4AC08091D0028F7D46C0809110
:1041C000D0028F7B42C08091D002877F8B7F3DC021
:1041D0008091D1028D7F8E7F15C08091D00282FBAD
:1041E000222720F991E0922790FB82F990FB83F936
:1041F0002CC08091D102982F909591708E7F892B41
:1042000090FB81F98093D10222C00E94DD0780914A
:10421000D00287FB222720F991E0922790FB87F9B3
:1042200014C081E00E94BD0E12C08091D00284FBB8
:10423000222720F991E0922790FB84F906C0809113
:10424000D002982F909590FB80F98093D0028091B6
:10425000D0029091D1020E94370E0E94DD0780E0CB
:1042600001C081E0DF91CF910895893279F1E0F4C6
:10427000843161F1A0F4873009F075C01092940286
:1042800094E190932201809321018CE3809320019B
:1042900088E080931E0188E280931D0164C092EE45
:1042A000980F9A30F0F05FC0803509F444C028F4CC
:1042B0008F3409F058C08AE03FC0813529F082353B
:1042C00009F051C081E038C08FEF36C08091B00254
:1042D000882379F11092B0021092AF021092AE02D0
:1042E00042C08D518093B002833099F038F4813010
:1042F00069F08230D9F482E291E00DC0853099F006
:1043000078F0863099F48DE191E005C084E992E07F
:1043100002C081E291E09093AF028093AE0223C08D
:1043200080E291E0F8CF8EE191E0F5CF1092B002FB
:104330001AC080E0089586EFE091AE02F091AF02DE
:10434000309789F02081082E000C990B820F911D67
:104350008F3F910519F014F08FEF04C097FF02C052
:10436000108201C0808381E008950F931F9341E084
:1043700050E060E070E08A019B0104C0000F111F53
:10438000221F331F8A95D2F7C901B8010E94350850
:104390001F910F910C94DD078B3109F468C058F51B
:1043A0008B3009F486C078F4863009F445C020F4D7
:1043B000853009F44BC07FC0873009F44AC088308B
:1043C00009F477C078C0803109F464C068F48E3095
:1043D00009F071C080916F0282FB222720F991E0E1
:1043E000922790FB82F94CC0863109F462C0893172
:1043F00009F45FC060C08A32E1F060F4873209F4EA
:1044000055C028F48E3108F456C08D5150C0893201
:10441000E9F051C0833450F48A3308F045C0853345
:1044200009F444C0883309F444C045C08334F1F131
:1044300042C00E94BB0E3DC080916F02817F8E7F83
:1044400080936F0281E08093B10208950E9420035F
:1044500030C080916F02982F9095917090FB80F9F9
:1044600080936F02911125C0897F877F10C0809152
:104470006F0281FB222720F991E0922790FB81F9BE
:1044800080936F029923A9F080916F0281608093DD
:104490006F020FC080916F0283FB222720F991E009
:1044A000922790FB83F9ECCF895301C080E00E94F2
:1044B000B52181E0089580E0089580E008950C948E
:1044C0005D22CF93C82F8091B102813069F038F01E
:1044D0008230C1F58C2F0E94352181E039C00E94C5
:1044E000300D823289F504C00E94300D823261F4B1
:1044F0008C2F0E945F22811104C08C2F0E94CC213E
:104500001FC081E090E01CC08C2F0E945D228111B1
:1045100016C0C43189F058F4CB3089F0C031B1F401
:1045200082E08093B10288E30E94352108C0C9323D
:1045300019F0C83321F00AC01092B10207C081E01F
:10454000817006C01092B10280E002C080E0F8CF16
:10455000CF910895CF93DF9386319C4541F5EB01D0
:104560000E94300D982F8A81209102013091030121
:10457000882379F09A7A81E009F480E08093B2028E
:10458000911102C069E201C065E3C9010E940626DB
:104590000AC08091B202811102C069E201C065E3E4
:1045A000C9010E9408260E94720D80E001C081E0CE
:1045B000DF91CF9108950F931F93CF93DF93C42F73
:1045C000D22FFC0182818823C9F04093B5020E945A
:1045D000AC269093B4028093B30280E28C0F8830B3
:1045E00008F057C0C77081E001C0880FCA95EAF78C
:1045F000DF91CF911F910F910C943A058091B502F4
:10460000481330C08091B3029091B4020E94C42636
:10461000883C910538F510E21D0FCD17B9F080E206
:104620008C0F883040F4C77081E001C0880FCA95B4
:10463000EAF70E944105183028F581E09D2F977018
:1046400001C0880F9A95EAF70E943A05802F0E94D0
:1046500031051830F0F4D77081E001C0880FDA9589
:10466000EAF70AC080E28C0F883098F4C77081E0C6
:1046700001C0880FCA95EAF7DF91CF911F910F9182
:104680000C944105802FDF91CF911F910F910C94D5
:104690003105DF91CF911F910F9108950F939C01E8
:1046A000CB01243F4CE5340731F188F4293DFCE58A
:1046B0003F07D9F02A3D4CE5340779F1283D3C45C8
:1046C000A9F506E221EE41EE68ED7CE52BC0263F20
:1046D000FCE53F07E1F0A8F0273F3C4539F507E24C
:1046E00025EE46EE67EF7CE51DC007E225EE45EEC0
:1046F00069ED7CE517C006E221EE40EE64EF7CE553
:1047000011C007E225EE44EE65EF7CE50BC006E242
:1047100021EE42EE66EF7CE505C008E221E045EEC1
:104720006AED7CE50E94DB2280E008C0FC0182810A
:10473000882319F01092B50201C081E00F9108950D
:104740008EE1489B02C08150E1F7489BFECF08955F
:10475000589880E28A95F1F7589A0895FC012AE06A
:104760002A95F1F728E090E080E031E040E14A95B9
:10477000F1F7880F489B02C08160932700C00000BA
:1047800040E14A95F1F7215089F720E12A95F1F7A8
:1047900029B100C0000030E13A95F1F7217092276D
:1047A0002081920F90830895EF92FF920F931F93B1
:1047B000CF93DF931F92CDB7DEB719828C017C01B6
:1047C000E60EF11C0E151F0551F00E94A023CE012C
:1047D00001960E94AE23F80181938F01F3CF81E00F
:1047E0009981911180E00F90DF91CF911F910F91EE
:1047F000FF90EF900895509A589A08955098589ABB
:10480000E89AE9E6F0E080818C7F8083089561502A
:1048100091E001C0990F6A95EAF720E031E0992311
:1048200061F0492F482319F0589A232701C058985E
:1048300040E24A95F1F79695F2CF222311F0589A6B
:1048400001C0589880E28A95F1F758980895FF9230
:104850000F931F93CF93DF93EC018C01060F111D73
:10486000C017D10741F0F9900E94A82368E08F2D6E
:104870000E940724F5CFDF91CF911F910F91FF90F8
:1048800008951F920F920FB60F9211240F931F934A
:104890002F933F934F935F936F937F938F939F9348
:1048A000AF93BF93EF93FF93CF93DF931F92CDB757
:1048B000DEB719820E94A023CE0101960E94AE238A
:1048C000082F069506950695902F96959570202FA2
:1048D0002570920F292F237096959695920F8770C9
:1048E00089135FC0898181115CC0043008F059C010
:1048F00080E18A95F1F7589A509A82E08A95F1F70B
:1049000000C0589888E0089F80011124D801AB5F4F
:10491000BE4F1696ED91FC9117973097A9F06091D4
:10492000B1017091B20114962D913C911597260F0B
:10493000371F11968D919C911297680F791F1396CE
:104940004C9113978C910995F801EB5FFE4F6381B1
:10495000662351F08091B1019091B201248135819B
:10496000820F931F0E9427240E94A82380E18A952A
:10497000F1F758985098589A80E18A95F1F7F80124
:10498000EB5FFE4F6081662351F08091B101909101
:10499000B20121813281820F931F0E94D4230E9491
:1049A000A0230F90DF91CF91FF91EF91BF91AF9135
:1049B0009F918F917F916F915F914F913F912F9137
:1049C0001F910F910F900FBE0F901F9018950F938E
:1049D0001F93CF93DF93843091050CF06DC0EC01F1
:1049E000F894509A589885E08A95F1F700009C2F2A
:1049F000969595702C2F2570920F892F8370969520
:104A0000969523E0CC0FDD1F2A95E1F7980F8E01D4
:104A1000092B0E94A82384E08A95F1F700C068E082
:104A2000802F0E94072480E18A95F1F75098589AC8
:104A3000489902C000C0FCCF87E090E0489B08C0C6
:104A4000019721F4509A589A789436C000C0F6CF56
:104A5000FE01EB5FFE4F6381662381F08091B1011F
:104A60009091B20124813581820F931F0E94D4233B
:104A7000811104C0509A589A78941FC00E94A023B4
:104A800080E28A95F1F75898509A80E18A95F1F77B
:104A9000CB5FDE4F6881662351F08091B101909128
:104AA000B20129813A81820F931F0E9427240E941C
:104AB000A823789481E001C080E0DF91CF911F911D
:104AC0000F9108959093D9018093D8010895909300
:104AD000BC028093BB0208950E94DB13811103C0C6
:104AE0008091B6020895E091BB02F091BC0230972C
:104AF00021F00190F081E02D099480E00895E0918B
:104B0000BB02F091BC02309721F00280F381E02DCE
:104B100009940895E091BB02F091BC02309739F0FE
:104B200022E0DC012C930480F581E02D09940895A6
:104B30002091B9023091BA022817390771F0909389
:104B4000BA028093B902E091BB02F091BC023097A7
:104B500021F00680F781E02D099408952091B70295
:104B60003091B8022817390771F09093B8028093FA
:104B7000B702E091BB02F091BC02309721F00084B3
:104B8000F185E02D09940895FC01329697E080E0CC
:104B9000915029F021912223D9F38F5FF9CF089505
:104BA000662349F0FC01329608962191621729F09C
:104BB000E817F907D1F780E0089581E008959C0196
:104BC000FC0132969FEF80E04191461789F09F3FAC
:104BD00019F4411101C0982F8F5F8630A9F79F3FCC
:104BE00039F0F901E90FF11D97FDFA9562830895F7
:104BF00008959C012A5F3F4FFC014281461301C08A
:104C00001282019682179307B9F708950C94DF2555
:104C10000C94F925029626E0FC0111922A95E9F7F9
:104C2000089508950C94112683E08093BD020C949E
:104C30001226811102C081E001C082E08093BD0292
:104C40000C9412260C94192681E08093BD020C94DA
:104C500012260C94242608950C942B260C942C26B2
:104C60000C942B260C942B260C942B26CF930E946D
:104C700032260E9450130E943026C0E08C2F0E94E2
:104C80001112811104C0CF5FCA30C1F701C081E0A9
:104C9000CF91089508951F920F920FB60F9211248D
:104CA0008F939F93AF93BF938091BE02811113C0E6
:104CB0008091170390911803A0911903B0911A03E2
:104CC0004196A11DB11D8093170390931803A093E3
:104CD0001903B0931A03BF91AF919F918F910F90D9
:104CE0000FBE0F901F90189580911F03843031F1F3
:104CF0000E9488031092BE0220E488E190E00FB683
:104D0000F894A895809360000FBE2093600083B74D
:104D1000817F846083BF83B7816083BF78948895E7
:104D200083B78E7F83BF0FB6F894A89580916000FB
:104D3000886180936000109260000FBE08950E9409
:104D4000DD070C948C0382E084BD93E095BD9AEF5F
:104D500097BD80936E0008952FB7F8948091170344
:104D600090911803A0911903B0911A032FBF0895D1
:104D70002FB7F8946091170370911803809119036D
:104D800090911A032FBF08959C014FB7F89480911A
:104D9000170390911803A0911903B0911A034FBF04
:104DA000821B930B0895CF92DF92EF92FF922FB761
:104DB000F894C0901703D0901803E0901903F09076
:104DC0001A032FBFA7019601261B370B480B590B5F
:104DD000CA01B901FF90EF90DF90CF9008957894C9
:104DE0001F920F920FB60F9211248F939F93AF9340
:104DF000BF938091170390911803A0911903B0916C
:104E00001A030196A11DB11D8093170390931803F7
:104E1000A0931903B0931A03BF91AF919F918F9103
:104E20000F900FBE0F901F90189587E797E790930C
:104E30000108809300089AE088E10FB6F894A895DD
:104E4000809360000FBE90936000FFCF8091CA02F4
:104E50000895089522E02093E9002FEF3091E800B3
:104E6000215035FD06C035ED3A95F1F700002111CE
:104E7000F5CF2091E80025FF0BC040E050E066E050
:104E800070E00E9454298091E8008E778093E800BA
:104E90000895CF93DF9321E02093E9002FEF309125
:104EA000E800215035FD06C035ED3A95F1F70000D8
:104EB0002111F5CF2091E80025FF14C0EC0140E05E
:104EC00050E068E070E00E9454298091E8008E77FD
:104ED0008093E80088E0FE01A2ECB2E001900D9220
:104EE0008A95E1F7DF91CF9108958093BF02709387
:104EF000C1026093C00280911F03843001F582E0FB
:104F00008093E9008FEF9091E800815095FD06C0F5
:104F100095ED9A95F1F700008111F5CF8091E800A9
:104F200085FF0DC040E050E063E070E08FEB92E061
:104F30000E9454298091E8008E778093E8000895BC
:104F4000BC0184E00C947527BC0183E00C947527A8
:104F500080911E03811109C00E94E52A0E94422B04
:104F60008091E20084608093E200089510921E0315
:104F700008950C94292660911B0381E0611101C002
:104F800080E00C94142690911F0381E0943009F086
:104F900080E060911B030C94192642E061EC81E0F3
:104FA0000E945E2A42E261EC82E00E945E2A9091B9
:104FB0001F0381E0943009F080E060911B030C94A2
:104FC000222680912103833009F461C030F48130BE
:104FD00071F0823009F49AC008958A3009F486C0CD
:104FE0008B3009F46CC0893009F0A8C020C08091D2
:104FF0002003813A09F0A2C08091E800877F809366
:10500000E8008091240390912503892B21F468E026
:1050100082EC92E003C060E080E090E070E00E94EB
:105020009F298091E8008B778093E8000895809114
:105030002003813209F082C08091240390912503DE
:10504000029708F07BC08091E800877F8093E8009A
:105050008091E80082FD05C080911F038111F8CF87
:105060006DC02091F3008091F20090E0922B0297A6
:1050700031F48091F100813011F0863021F480917B
:10508000F1008093CA028091E8008B7753C0809131
:105090002003813A09F052C08091240390912503A6
:1050A000892B09F04BC08091E800877F8093E8004E
:1050B0008091E80080FFFCCF8091420136C0809152
:1050C00020038132D9F58091240390912503892B07
:1050D000A9F58091E800877F8093E8000E94932AD9
:1050E00080912203809342010C94DD07809120037C
:1050F000813221F58091E800877F8093E8000E944B
:10510000932A809123038093CB02089580912003FA
:10511000813AA1F48091E800877F8093E800809134
:10512000E80080FFFCCF8091CB028093F10080915A
:10513000E8008E778093E8000C94932A089584B752
:10514000877F84BF0FB6F894A8958091600088612E
:1051500080936000109260000FBE90E080E80FB670
:10516000F89480936100909361000FBE0C94242604
:105170000E94E52A0E94422BE2EEF0E080818460EA
:10518000808378940C94D72D86E391E00C94672566
:1051900080911F038530A9F480911F03853079F435
:1051A0000E94742680911D038823B1F30E94362645
:1051B000882391F30E943E290E94DD07EDCF0C94D5
:1051C0009F26089508950C94E528292F332723302E
:1051D0003105C9F060F42130310581F0223031050C
:1051E00009F044C08BE390E02BE434E043C021326B
:1051F0003105E1F02232310549F138C082E190E019
:1052000026E834E037C099278130910549F028F02D
:10521000029761F5E7E0F4E005C0E7E4F4E002C0DE
:10522000EFE2F4E0849190E09F0124C061157105E4
:1052300041F061307105D1F489E090E026E734E077
:1052400019C089E090E02DE534E014C061157105C6
:1052500041F06130710551F48BE790E028E934E0CA
:1052600009C080E490E023E135E004C080E090E0F4
:1052700020E030E0FA0131832083089580E189BD88
:1052800082E189BD09B400FEFDCF8091D8008F7DF9
:105290008093D8008091E00082608093E00080914C
:1052A000E00081FDFCCF0895CF92DF92EF92FF9254
:1052B0000F931F93CF93DF93EC018B017A010E9430
:1052C000B22A811133C0E114F10439F0F701808171
:1052D0009181081B190BC80FD91FC12CD12C0115A6
:1052E000110519F18091E80085FD16C08091E80054
:1052F0008E778093E800E114F10449F0F701808192
:105300009181C80ED91ED182C08285E00FC00E9453
:10531000B22A882321F30AC089918093F1000150B9
:105320001109FFEFCF1ADF0ADACF80E0DF91CF91CA
:105330001F910F91FF90EF90DF90CF9008952091F3
:105340002603309127032617370748F061157105AA
:1053500039F42091E8002E772093E80001C0B901CC
:10536000FC0120E06115710579F180911F0388230C
:10537000F1F18530F1F18091E80083FD3CC080912E
:10538000E80082FD2EC08091E80080FFEBCF2091E5
:10539000F3008091F20090E0922B6115710551F0BD
:1053A0008830910538F421912093F1006150710902
:1053B0000196F3CF21E0089709F020E08091E80002
:1053C0008E778093E800CECF2111CFCF0AC0809195
:1053D0001F03882361F0853061F08091E80083FD30
:1053E0000AC08091E80082FFF2CF80E0089582E059
:1053F000089583E0089581E0089520912603309177
:1054000027032617370748F06115710539F42091F5
:10541000E8002E772093E80001C0B901FC0120E0EC
:105420006115710591F180911F03882309F440C033
:10543000853009F43FC08091E80083FD3DC0809134
:10544000E80082FD2FC08091E80080FFE9CF209125
:10545000F3008091F20090E0922B6115710559F0F4
:105460008830910540F424912093F10031966150E9
:1054700071090196F2CF21E0089709F020E08091B0
:10548000E8008E778093E800CBCF2111CCCF0AC003
:1054900080911F03882361F0853061F08091E800DE
:1054A00083FD0AC08091E80082FFF2CF80E008957A
:1054B00082E0089583E0089581E00895982F973061
:1054C00068F59093E900981739F07091EC002091FD
:1054D000ED005091F00003C0242F762F50E021FD05
:1054E00002C09F5FECCF3091EB003E7F3093EB002A
:1054F0003091ED003D7F3093ED003091EB00316055
:105500003093EB007093EC002093ED005093F0008B
:105510002091EE0027FDE5CF80E008958F70809305
:10552000E90081E008958091200387FF11C08091F8
:10553000E80082FD05C080911F038111F8CF11C0E2
:105540008091E8008B770BC080911F03882349F07E
:105550008091E80080FFF8CF8091E8008E778093FB
:10556000E80008952091E4003091E50095E640912F
:10557000EC00842F817040FF23C08091E80080FD03
:105580001DC080911F03882399F0853099F0809188
:10559000EB0085FD11C04091E4005091E500241717
:1055A000350729F3915011F09A01E1CF84E0089575
:1055B00082E0089583E0089581E0089580E00895F1
:1055C0004091E80042FFDDCF08950E94532B0E94D6
:1055D0005B2BE0EEF0E0808181608083E8EDF0E01D
:1055E00080818F77808319BCA7EDB0E08C918E7F8E
:1055F0008C9380818F7E808310921E0308950F9379
:105600001F93CF93DF930E94532B0E945B2BC8ED17
:10561000D0E088818F7788838881806888838881BB
:105620008F7D888319BC10921F0310921B03109268
:105630001D0310921C0300EE10E0F80180818B7FA7
:10564000808388818160888342E060E080E00E94FE
:105650005E2AE1EEF0E080818E7F8083E2EEF0E072
:10566000808181608083808188608083F80180816F
:105670008E7F8083888180618883DF91CF911F91A5
:105680000F910895E8EDF0E080818F7E8083E7ED53
:10569000F0E080818160808384E082BF81E080933C
:1056A0001E030C94FF2AE8EDF0E080818E7F80835A
:1056B0001092E20008951092DA001092E10008952D
:1056C0001F920F920FB60F9211242F933F934F9377
:1056D0005F936F937F938F939F93AF93BF93EF935A
:1056E000FF938091E10082FF0BC08091E20082FF76
:1056F00007C08091E1008B7F8093E1000E94D62D4E
:105700008091DA0080FF1FC08091D80080FF1BC00D
:105710008091DA008E7F8093DA008091D90080FF3B
:105720000DC080E189BD82E189BD09B400FEFDCFD5
:1057300081E080931F030E94A82705C019BC109226
:105740001F030E94B6278091E10080FF19C080915D
:10575000E20080FF15C08091E2008E7F8093E2001E
:105760008091E20080618093E2008091D8008062A5
:105770008093D80019BC85E080931F030E94BB274B
:105780008091E10084FF30C08091E20084FF2CC052
:1057900080E189BD82E189BD09B400FEFDCF809121
:1057A000D8008F7D8093D8008091E1008F7E809318
:1057B000E1008091E2008F7E8093E2008091E20020
:1057C00081608093E20080911B03882311F084E0C4
:1057D00007C08091E30087FD02C081E001C083E043
:1057E00080931F030E94C3278091E10083FF29C09B
:1057F0008091E20083FF25C08091E100877F809344
:10580000E10082E080931F0310921B038091E1006E
:105810008E7F8093E1008091E2008E7F8093E20092
:105820008091E20080618093E20042E060E080E0ED
:105830000E945E2A8091F00088608093F0000E94B0
:10584000B927FF91EF91BF91AF919F918F917F9178
:105850006F915F914F913F912F910F900FBE0F90DD
:105860001F9018951F920F920FB60F9211242F932D
:105870003F934F935F936F937F938F939F93AF93D8
:10588000BF93CF93DF93EF93FF93C091E900CF7065
:105890008091EC00D82FD17080FDD0E81092E90003
:1058A0008091F000877F8093F00078940E94762C9E
:1058B0001092E9008091F00088608093F000CD2B79
:1058C000CF70C093E900FF91EF91DF91CF91BF912D
:1058D000AF919F918F917F916F915F914F913F9188
:1058E0002F910F900FBE0F901F9018951F93CF937D
:1058F000DF93CDB7DEB7AA970FB6F894DEBF0FBE21
:10590000CDBFE0E2F3E08091F100819323E0E83243
:10591000F207C9F70E94E1278091E80083FF2EC1BA
:105920008091200390912103492F50E04A30510586
:1059300008F024C1FA01EE59FF4F0C945C2E803818
:1059400021F0823809F01AC108C080911C0390919F
:105950001D03992389F082600FC0809124038F700A
:10596000873008F00BC18093E9008091EB0085FB44
:10597000882780F91092E9009091E800977F909332
:10598000E8008093F1001092F100D1C0282F2D7F04
:1059900009F0F4C0882319F0823061F0EFC08091E3
:1059A0002203813009F0EAC0933009F080E080934F
:1059B0001D032EC08091220381112AC080912403EF
:1059C0008F702FEF280F263008F0D8C08093E900A1
:1059D0002091EB0020FF1CC0933021F48091EB005C
:1059E000806214C09091EB0090619093EB0021E0F5
:1059F00030E0A90102C0440F551F8A95E2F7409399
:105A0000EA001092EA008091EB0088608093EB003E
:105A10001092E9008091E800877F8093E8000E945F
:105A2000932AACC08111AAC0109122031F778091E4
:105A3000E3008078812B8093E3008091E800877FEA
:105A40008093E8000E94932A8091E80080FFFCCFB9
:105A50008091E30080688093E300111102C082E02E
:105A600001C083E080931F0389C08058823008F012
:105A700085C080912203909123038C3D53E09507CC
:105A800079F583E08A838AE289834FB7F894DE014F
:105A9000139620E03EE051E2E32FF0E050935700F0
:105AA000E49120FF03C0E295EF703F5FEF708E2F0F
:105AB00090E0EA3010F0C79601C0C0968D939D9398
:105AC0002F5F243149F74FBF8091E800877F809393
:105AD000E8006AE270E0CE0101960E949F2916C09C
:105AE0006091240370912503AE014F5F5F4F0E94C8
:105AF000E328BC01892B09F441C09091E800977F0D
:105B00009093E80089819A810E94FD298091E800A4
:105B10008B778093E80032C0803881F58091E8006F
:105B2000877F8093E80080911B038093F100809130
:105B3000E8008E7772CF811121C08091220390916D
:105B4000230399270297D4F48091E800877F8093FC
:105B5000E8008091220380931B030E94932A809186
:105B60001B03811106C08091E30087FD02C081E024
:105B700001C084E080931F030E94CD278091E8003C
:105B800083FF0AC08091E800877F8093E8008091BE
:105B9000EB0080628093EB00AA960FB6F894DEBF0C
:105BA0000FBECDBFDF91CF911F9108950895CF9380
:105BB00080911F038823A1F0C091E900CF709091DC
:105BC000EC00892F817090FD80E8C82B1092E900CD
:105BD0008091E80083FD0E94762CCF70C093E9008D
:105BE000CF9108950E94E52A10921F030895E8EDD1
:105BF000F0E08081806180838AE18A95F1F700C0BE
:105C00008091D9008170089587FB082E062687FDB4
:105C1000819567FD61950E94932E0EF4919507FC86
:105C200081950895AA1BBB1B51E107C0AA1FBB1F8A
:105C3000A617B70710F0A61BB70B881F991F5A9518
:105C4000A9F780959095BC01CD01089597FB072E8B
:105C500016F4009407D077FD09D00E94122E07FC9D
:105C600005D03EF4909581959F4F0895709561956C
:105C70007F4F0895A1E21A2EAA1BBB1BFD010DC088
:105C8000AA1FBB1FEE1FFF1FA217B307E407F507EC
:105C900020F0A21BB30BE40BF50B661F771F881FC8
:105CA000991F1A9469F760957095809590959B015E
:105CB000AC01BD01CF010895EE0FFF1F0590F491D7
:105CC000E02D09940E946A2E332312F48A1B9B0B49
:105CD0000C947B2EA29FB001B39FC001A39F700DB7
:105CE000811D1124911DB29F700D811D1124911DE4
:105CF00008950E946A2EB7FF0895821B930B0895A2
:105D00000E946A2EA59F900DB49F900DA49F800DB8
:105D1000911D11240895B7FF0C94802E0E94802EAF
:105D2000821B930B0895991B79E004C0991F961765
:105D300008F0961B881F7A95C9F780950895FC0195
:105D40004150504030F001900616D1F73197CF0105
:105D50000895882799270895FB01DC0104C08D91DF
:105D60000190801921F441505040C8F7881B990BCD
:105D70000895FB01DC0102C001900D92415050409A
:105D8000D8F70895F999FECF92BD81BDF89A992769
:105D900080B50895A6E1B0E044E050E00C94FC2EFC
:105DA000A8E1B0E042E050E00C94FC2E262FF999D7
:105DB000FECF92BD81BDF89A019700B4021639F06A
:105DC0001FBA20BD0FB6F894FA9AF99A0FBE08953B
:105DD0000396272F0E94D72E0E94D62E252F0E9491
:105DE000D72E242F0C94D72E0196272F0E94D72E22
:105DF0000C94D62EDC01CB01FC01F999FECF06C034
:105E0000F2BDE1BDF89A319600B40D924150504078
:085E1000B8F70895F894FFCFE4
:105E1800C80053020100000001000000000000005B
:105E280005010000000406000000000000280850DA
:105E38003C0714010102000E000E0E01191A1B1C6A
:105E48001D1E1F202122262749272A27A427A027ED
:105E5800292701E200E900EA00B500B600B700CD45
:105E6800008301CC008A01920194012102230224BB
:105E7800022502260227022A02B300B4006F00702E
:105E880000818283E200E900EA00B500B600B700AD
:105E9800CD008301CC008A019201940121022302E2
:105EA80024022502260227022A02B300B4006F004A
:105EB8007000818283F5F6F7313332369497C63411
:105EC80035780200010202020206060609090909DC
:105ED80009090F0F0F0F0F0F151515181919191993
:085EE8001919191919192324D5
:00000001FF
